:020000040000FA
:04000000803119280A
:100008007E1480310B1F09280A2817282100101F89
:100018000E280F2817282000101F13281428172827
:100028008131742180317E10090080311B28F20152
:10003800F3017E1020008131562920000E1E25284C
:1000480026284928A0309B00A03028009500E430DD
:1000580021001C02031C312832283428E3309C007C
:100068001B301C02031839283A283C281B309C00F6
:100078001C08EA3E2800940020008E1A44284528CF
:100088006B286930280094006B287A309B00B030C8
:1000980028009500FD3021001C02031C5428552817
:1000A8005728FC309C0002301C0203185C285D288D
:1000B8005F2802309C001C08013E280094002000A4
:1000C8008E1A672868286B2880302800940006302C
:1000D8003E00AF000230AF00080022008C018E0104
:1000E800333021008C0039308E00013023008E001F
:1000F80011308C000A3024008C0039308E00210029
:10010800951325008C018E01373026008C003F3076
:100118008E003F3027008C003F308E0006303D00B7
:10012800A00002303C0093001430A80007303D00C6
:10013800A1000530A200043092000800803171202F
:10014800803181318A2180318031FD2080318131B7
:1001580036218031813124218031813182218031E1
:100168008131652180318031C4208031813146213F
:1001780080318131112180318031E42080310800C3
:1001880028009701113096000530980080309400BF
:1001980020000E1ED028D128D428693028009400C9
:1001A8002800930120009110B0302800950020000D
:1001B8000E1EDF28E028E328A0302800950008005C
:1001C80020008C1CE828E928EC2880309900ED28CC
:1001D80099019701960110101708F3001608F2000C
:1001E800143098008E1DF928FA28FC28043098004D
:1001F800080005303E0091000C3092000430930056
:100208001A3094000730950009309600970198013C
:1002180080309900A3309000080020009E01113022
:100228009D0003309F007A309B000E1E1C291D295B
:100238001F29A0309B009A019010C0309C00080034
:10024800103021009E0040309F009B019C0101302E
:100258009D0010172130F4000030F5008131912104
:100268008131080006303E00AF001A30B000B101FD
:10027800B201B3010230B400B501B601B701A43030
:10028800AE00080002303E009B000C309C009D012F
:100298009E019F010230A000A101A201A301A0308C
:1002A8009A0008008031A220813120001814013002
:1002B8003E0091000230AF008B170B176229803186
:1002C800192882303E00A500A601A701A801A901AE
:1002D8000230AA00AB01AC01AD01A030A4000800B7
:1002E800200010137008710403197B297C298129C7
:1002F80071088A0070080A00813108008B302500D7
:1003080093009C3092003F30910008003830210063
:10031800990098012200960108007508F1007408F8
:04032800F0000800D9
:020000040001F9
:06000E00FA3FFF1E9F3FB8
:00000001FF
